:100000008317753084007E300A128A110D200A127F
:100010008A1183010A128A11152864008001840A5A
:1000200004060319003404060E280A168A116B20F0
:100030000A128A11003083120313C8000030C9006D
:1000400000300A128A11DE270A128A110030831248
:100050000313A0000030A1002D28CB010314CB0D09
:100060000C302007840002300318033021070A12E5
:100070008A1100220A128A110A168A11AC220A1267
:100080008A11831203130130A0070318A10A00305C
:10009000A1072108803AA20081302202031D5228C4
:1000A000F8302002031C552856282D280530C8009A
:1000B0000030C90028300A128A11DE270A128A117C
:1000C000D73083120313C0000730C1000A128A110F
:1000D000BB200A128A11C83083120313C9000030F2
:1000E000CA000A168A1153200A128A110A168A11A6
:1000F0001B270A128A110A168A11F8200A128A117D
:1001000083120313061C852886288C280A128A1558
:1001100042230A128A1191280A128A158D250A1281
:100120008A1101300A168A114D220A128A111E30D4
:1001300083120313C9000030CA000A168A11532023
:100140000A128A1100300A168A114D220A128A11E7
:10015000143083120313C9000030CA000A168A1132
:0E01600053200A128A1180280A128A110028E0
:10017600D2284008840041080A128A1100220A1275
:100186008A110A128A15AB200A128A1101308312CB
:100196000313C0070318C10AC200C21BC1034008EB
:1001A600840041080A128A1100220A128A110038B4
:1001B600031DDE28DF28BC280800E1284D30CF00CB
:1001C60043300A168A11F3210A128A118312031385
:1001D600CB00CD08031DF028F128F8284608C300F7
:1001E6004708C4004808C500FF294C30CF004630F8
:1001F6000A168A11F3210A128A1183120313C900FF
:10020600CC08031D0729ED290630CA004C088313C4
:100216004D0203180F2910294F294C08CE004D080E
:10022600CE0219304E02031C19291A29252900303D
:10023600C3000030C4000030C5004C08CD0049089A
:10024600CB004E2901300310C60DC70DC80DFF3E69
:10025600031D26290130CC024C084D06031934290A
:1002660035293B290130CA02031D3A293B29252994
:10027600482901300310C50CC40CC30CFF3E031DF6
:100286003D290130CE004E08CD074D084C06031D12
:100296004D294E293C298F294D084C06031954290E
:1002A60055298F294D08CE004C08CE0219304E0232
:1002B600031C5E295F2966290030C6000030C7008E
:1002C6000030C8008F2901300310C30DC40DC50DC1
:1002D600FF3E031D67290130CD024C084D06031968
:1002E600752976297C290130CA02031D7B297C29C0
:1002F6006629892901300310C80CC70CC60CFF3EBD
:10030600031D7E290130CE004E08CC074D084C0651
:10031600031D8E298F297D29CB08031D9329A72923
:10032600FF30C306FF30C406FF30C5060130C307E1
:10033600003003110318013E031DC40700300311EA
:100346000318013E031DC507C908031DAB29BF29B4
:10035600FF30C606FF30C706FF30C8060130C607A5
:10036600003003110318013E031DC70700300311B7
:100376000318013E031DC80703100030031801309F
:10038600CB004608C307470803110318470A031D95
:10039600C407480803110318480A031DC507C51FEB
:1003A600D529D629ED29FF30C306FF30C406FF3014
:1003B600C5060130C307003003110318013E031DB3
:1003C600C407003003110318013E031DC507CB0106
:1003D6000314CB0D4D088313CF0043300A168A1140
:1003E60045260A128A1183120313CB08031DFC2922
:1003F600FE298030C506FF290800FE00FE1F082AD8
:1004060083137E188317000808008A0004088200F8
:10041600003400344034C034C03480348034003476
:100426000034003400340034003400340034003426
:100436000034003400340034003400340034003416
:100446000034003400340034003400340034003406
:1004560000340034003400340034003400340034F6
:1004660000340034003400340034003400340034E6
:10047600003400340034003400340034E034F834FE
:10048600F034E0340034003400340034E034E03436
:10049600E034C034803410347C34FC34FE34FC3414
:1004A600F834E034C034003400340034003400340E
:1004B6000034003400340034003400340034013495
:1004C60007341F347F34FC34F834E034803400348D
:1004D600003400340034FC34FE34FC34DC3418348C
:1004E60038347034E034803400340034003400345E
:1004F60000340034003400340034003480340034D6
:10050600003480348034803400348034C034C034C5
:10051600C0348034803400340034F034F834F83495
:1005260078347034F034CF349F343F347F34FF3422
:10053600F634C03487347F34FF34FF34E7349F34D5
:10054600FC34FB34FF34FF34FF34FF34FF34DF3434
:1005560018340034003400340034003400340034DD
:1005660000340034003400340034003400340134E4
:1005760003340F347F34FE34F834E03480340034EE
:1005860007343F34FF34FE34FC34E03401340334A2
:100596000F340434003400340034003400340034A2
:1005A60003340F343F34FF34FF34FF34E7341F3451
:1005B6007F34FF34FF34F334CF343F34FF34FE341A
:1005C600F834E3349F347F34FF34FC34FF34DF34B3
:1005D6001F340F340E34C334CF343F34FF34FE346B
:1005E600F934C7341F347F34FF34FF34F334833493
:1005F60003342134E734DF34FF34FC34F034C034C0
:100606000034003400340034003400340034003444
:100616000034003400340034003400340034013433
:1006260003340F343F34FE34F834E034803401347C
:1006360007341F34FF34FE34F834E0348034003499
:1006460004341C34F834F03480340034003401347B
:1006560003340F343F34FF34FE34F934E7349F3427
:100666007F347F347C34713407343F343F341E3456
:100676001D340134033407340F340E340E340C3475
:100686000F340F3400340134033407340F340E347E
:100696000F340734033407340E341E343D343F34EC
:1006A6003F34193407341F347F347E347834C034F1
:1006B6000034003400340034003400340034003494
:1006C6000034003400340034003400340034003484
:1006D60003340F343F34FE34F834F03480340134BC
:1006E60007340F349F34FF347C34F834F034F73455
:1006F600FF347E34003400340034003400340034D7
:100706000134013400340034003400340034003441
:100716000034003400340034003400340034003433
:100726000034003400340034003400340034003423
:100736000034003400340034003400340034003413
:100746000034003400340034003400340034003403
:1007560000340034003400340034003400340034F3
:1007660000340034003400340034003400340034E3
:1007760000340034003400340034003400340034D3
:1007860003340F343F34FE34FE347F343F341F3499
:100796000C340034003400340034003400340034A7
:1007A60000340034003400340034003400340034A3
:1007B6000034003400340034003400340034003493
:1007C6000034003400340034003400340034003483
:1007D6000034003400340034003400340034003473
:1007E6000034003400340034003400340034003463
:1007F6000034003400340034003400340034003453
:100806000034003400340034003400340034003442
:100816002F340034003400340734003407340034F5
:1008260014347F3414347F34143424342A347F341B
:100836002A3412342334133408346434623436349C
:1008460049345534223450340034053403340034EA
:10085600003400341C342234413400340034413432
:1008660022341C340034143408343E34083414342E
:10087600083408343E340834083400340034503424
:100886003034003410341034103410341034003442
:1008960060346034003400342034103408340434B6
:1008A60002343E345134493445343E340034423403
:1008B6007F34403400344234613451344934463450
:1008C6002134413445344B34313418341434123421
:1008D6007F341034273445344534453439343C3478
:1008E6004A344934493430340134713409340534D6
:1008F60003343634493449344934363406344934B9
:10090600493429341E340034363436340034003445
:100916000034563436340034003408341434223467
:10092600413400341434143414341434143400347C
:100936004134223414340834023401345134093435
:10094600063432344934593451343E347E34113409
:10095600113411347E347F344934493449343634C1
:100966003E3441344134413422347F3441344134BD
:1009760022341C347F3449344934493441347F3479
:1009860009340934093401343E3441344934493494
:100996007A347F340834083408347F3400344134E0
:1009A6007F34413400342034403441343F34013400
:1009B6007F3408341434223441347F344034403494
:1009C600403440347F3402340C3402347F347F3474
:1009D6000434083410347F343E34413441344134D5
:1009E6003E347F3409340934093406343E34413404
:1009F600513421345E347F34093419342934463471
:100A060046344934493449343134013401347F346D
:100A1600013401343F344034403440343F341F34D1
:100A26002034403420341F343F344034383440348A
:100A36003F346334143408341434633407340834CC
:100A460070340834073461345134493445344334FE
:100A560000347F3441344134003455342A3455341B
:100A66002A3455340034413441347F34003404345C
:100A760002340134023404344034403440344034C7
:100A86004034003401340234043400342034543405
:100A96005434543478347F34483444344434383409
:100AA60038344434443444342034383444344434BC
:100AB60048347F3438345434543454341834083475
:100AC6007E340934013402340C34523452345234F4
:100AD6003E347F34083404340434783400344434E7
:100AE6007D34403400342034403444343D340034C2
:100AF6007F341034283444340034003441347F3495
:100B0600403400347C3404341834043478347C346F
:100B160008340434043478343834443444344434A3
:100B260038347C341434143414340834083414340B
:100B3600143418347C347C340834043404340834D3
:100B46004834543454345434203404343F34443414
:100B5600403420343C344034403420347C341C341B
:100B66002034403420341C343C3440343034403457
:100B76003C34443428341034283444340C3450344F
:100B8600503450343C344434643454344C34443457
:100B960000340034003400340034003400340034AF
:100BA600003400340034FC34FC34C034C034C03467
:100BB600FC34FC3400340034003400340034003497
:100BC600003400340034003400341F341F34003441
:100BD600003400341F341F34E034E034C034603451
:100BE600E034E034C0346034E034C0340034FC34E3
:100BF600FC34C034C034C034FC34FC341F341F34DD
:100C0600003400341F341F34003400341F341F34C2
:100C160000341F341F340034003400341F341F34B2
:100C2600003400340034E034E03400340034E0347E
:100C3600E03400340034FC34FC34C034C034C034F6
:100C4600FC34FC34003400340034FF34FF341834F0
:100C560008341F341F34003400341F341F3400346A
:100C6600003400341F341F34003400340034E034C0
:100C7600E034C0346034E034C03400340034FC3432
:100C8600FC34C034C034C034FC34FC34003400348A
:100C960000341F341F34003400341F341F34003432
:100CA60000341F341F340034003400341F341F3422
:100CB600E034E034C0346034E034E034C0346034CE
:100CC600E034C03400340034FC34FC34CC34CC344E
:100CD600CC340C341F341F34003400341F341F341A
:100CE600003400341F341F34003400341F341F34E2
:100CF600003400340034003400340034003400344E
:100D0600E034E03400340034E034E03400340034BD
:100D1600FC34FC34CC34CC34CC340C3400340034C5
:100D260000340034FF34FF34183408341F341F34C1
:100D3600003400341F341F340034003400340034CF
:100D46000034003400340034E034E034C03460341D
:100D5600E034C03400340034FC34FC34CC34CC34BD
:100D6600CC340C3400340034003400341F341F34C7
:100D7600003400341F341F34003400341F341F3451
:100D860000340034003400340034003400340034BD
:100D9600E034E03460346034E034C034003400348D
:100DA600FC34FC34CC34CC34CC340C340034003435
:100DB60000340034FF34FF34183418341F34073439
:100DC600003400341F341F3400340034003400343F
:100DD600FC34FE34FE3406340634FE34FE34FC3471
:100DE6007F34FF34FF34C034C034FF34FF347F34E3
:100DF600003418341C34FE34FE34FE34003400341F
:100E060000340034C034FF34FF34FF34C0340034BF
:100E16003C343E343E3406348634FE34FE347C3470
:100E2600E034F034FC34FF34CF34C734C134C0343A
:100E36001C341E349E3486348634FE34FE34FC3430
:100E46007834F834F934C134C134FF34FF347E3495
:100E56000034F034FE347E34FE34FE34FE34003486
:100E66003F343F3437343034FF34FF34FF343034CA
:100E7600FE34FE34FE34C634C634C634C634863434
:100E86007134F134F134C034C034FF34FF347F346C
:100E9600FC34FE34FE34C634C634DE34DE349C34D0
:100EA6007F34FF34FF34C034C034FF34FF347F3422
:100EB6000634063406348634E634FE347E341E3474
:100EC6008034F034FE343F340734013400340034C7
:100ED6007C34FE34FE3486348634FE34FE347C3470
:100EE6007E34FF34FF34C134C134FF34FF347E34E2
:100EF600FC34FE34FE3486348634FE34FE34FC3450
:100F06007834F934F934C134C134FF34FF347F34D2
:100F16003834FE34823482348234823482348234E9
:100F26008234823482348234FE3470346C346534D4
:100F360061347334653420347734613469347434FD
:100F46002E342E340034203469346E3464347534CF
:100F56006334743461346E3463346534203400345D
:100F6600433461346C3469346234723461347434B9
:100F760069346E3467342E3400342034633461347B
:100F86007034613463346934743461346E34633478
:100F96006534003420342034203420342034203486
:100FA6002034203420340034593455345334273413
:100FB600303439340034CA000310003003180130CD
:100FC600CB004A08831380380A168A11AC220A120B
:100FD6008A11031083120313003003180130CB006B
:100FE60048088313073940380A168A11AC220A12B8
:040FF6008A11080054
:101016000030C6000030C7000030C8004430CF00A2
:101026003D300A168A11F3210A128A158312031318
:10103600C3004530CF0040300A168A11F3210A1248
:101046008A1583120313C9004908C306C508031D80
:101056002D283228C408031D31283228392846088D
:10106600BD004708BE004808BF00AA2845088313EC
:101076007B3EC9004908C4070730C5003D1C44280B
:10108600452853284008C607410803110318410A9A
:10109600031DC707420803110318420A031DC807A8
:1010A60001300310BF0CBE0CBD0CFF3E031D5428BF
:1010B60001300310C00DC10DC20DFF3E031D5C289B
:1010C6000130C502031D6828692841280930C5007A
:1010D6003D1C6E286F287D284008C607410803116D
:1010E6000318410A031DC707420803110318420AE1
:1010F600031DC80701300310BF0CBE0CBD0CFF3E1C
:10110600031D7E2801300310C80CC70CC60CFF3E19
:10111600031D86280130C502031D922893286B28DB
:1011260044088313CF0046300A168A1145260A1250
:101136008A1583120313C308031DA228A328C81700
:101146004608BD004708BE004808BF00AA28080098
:10115600C3007B3043020318B128B228B8282030D8
:1011660043020318B728B828B928C3290530CA008E
:101176000030CB00E030C400FF30C50043088313C5
:101186004407C80045080318450AC9000A168A110B
:10119600A4200A128A150430831203134807840018
:1011A60004300318053049070A128A1100220A1270
:1011B6008A15CB010314CB0D0A168A11AC220A122A
:1011C6008A15053083120313CA000030CB00E030C5
:1011D600C400FF30C500430883134407C800450810
:1011E6000318450AC9000A168A11A4200A128A158C
:1011F600831203134808013EC60049080318013E3E
:10120600003EC7000430460784000430031805304A
:1012160047070A128A1100220A128A15CB01031403
:10122600CB0D0A168A11AC220A128A1505308312D2
:101236000313CA000030CB00E030C400FF30C50005
:10124600430883134407C80045080318450AC90024
:101256000A168A11A4200A128A1583120313480853
:10126600023EC60049080318013E003EC70004308E
:101276004607840004300318053047070A128A110E
:1012860000220A128A15CB010314CB0D0A168A1105
:10129600AC220A128A15053083120313CA000030E5
:1012A600CB00E030C400FF30C50043088313440779
:1012B600C80045080318450AC9000A168A11A42061
:1012C6000A128A15831203134808033EC60049080A
:1012D6000318013E003EC700043046078400043070
:1012E6000318053047070A128A1100220A128A15C6
:1012F600CB010314CB0D0A168A11AC220A128A15E9
:10130600053083120313CA000030CB00E030C4005E
:10131600FF30C500430883134407C8004508031877
:10132600450AC9000A168A11A4200A128A158312D0
:1013360003134808043EC60049080318013E003E50
:10134600C7000430460784000430031805304707F9
:101356000A128A1100220A128A15CB010314CB0D38
:101366000A168A11AC220A128A1583120313CB01BC
:101376000314CB0D00300A168A11AC220A128A1504
:1013860008000230C8000030C90000300A128A1175
:10139600DE270A128A15CD3083120313C0000730E8
:1013A600C1000A128A11BB200A128A150330831261
:1013B6000313C8000030C90000300A128A11DE2764
:1013C6000A128A15CD3083120313C0000730C100FC
:1013D6000A128A11BB200A128A15033083120313DC
:1013E600C8000030C90023300A128A11DE270A120B
:1013F6008A1583120313CB010314CB0D70300A1622
:101406008A11AC220A128A1583120313CB01031424
:10141600CB0D70300A168A11AC220A128A15831275
:101426000313CB010314CB0D70300A168A11AC22BC
:101436000A128A15103083120313C2002730C30024
:101446003D08C001C0073E08C101C1070A168A113E
:10145600A9210A128A1583120313410840040319AD
:10146600352A362A532A1030C2002730C3003D08D9
:10147600C001C0073E08C101C1070A168A11A92189
:101486000A128A15831203134008BF003F08C100E1
:101496000530C00003300A168A1195250A128A15EE
:1014A600E83083120313C2000330C3003D08C001B5
:1014B600C0073E08C101C1070A168A11A9210A12EE
:1014C6008A15831203134008C001C0074108C101F1
:1014D600C1070A30C2000030C3000A168A1127214C
:1014E6000A128A158312031341084004031D7C2A3D
:1014F6007D2A942A1030C2002730C3003D08C0015F
:10150600C0073E08C101C1070A168A11A9210A129D
:101516008A1583120313410840040319932A942A57
:10152600C22AE830C2000330C3003D08C001C0072C
:101536003E08C101C1070A168A11A9210A128A1595
:10154600831203134008C001C0074108C101C10747
:101556000A30C2000030C3000A168A1127210A1277
:101566008A15831203134008BF003F08C1000F30DD
:10157600C00003300A168A1195250A128A156430AE
:1015860083120313C2000030C3003D08C001C00728
:101596003E08C101C1070A168A11A9210A128A1535
:1015A600831203134008C001C0074108C101C107E7
:1015B6000A30C2000030C3000A168A1127210A1217
:1015C6008A15831203134008BF003F08C100193073
:1015D600C00003300A168A1195250A128A150A30A8
:1015E60083120313C2000030C3003D08C001C007C8
:1015F6003E08C101C1070A168A11A9210A128A15D5
:10160600831203134008C001C0074108C101C10786
:101616000A30C2000030C3000A168A1127210A12B6
:101626008A15831203134008BF003F08C100283003
:10163600C00003300A168A1195250A128A150A3047
:1016460083120313C2000030C3003D08C001C00767
:101656003E08C101C1070A168A1127210A128A15F6
:10166600831203134008BF003F08C1003230C00098
:1016760003300A168A1195250A128A1508000530C4
:10168600C8000030C90007300A128A11DE270A1284
:101696008A15C03083120313C0000730C1000A1236
:1016A6008A11BB200A128A150A168A11FA230A120F
:1016B6008A15831203133D08B801B8073E08B9011D
:1016C600B9073808BD01BD073908BE01BE070A16AD
:1016D6008A11CE200A128A15831203133D08FB00D5
:1016E6003E08FC003F08FD007B08C0007C08C100E6
:1016F6007D08C2007508BD007608BE007708BF00E9
:101706000A168A115F210A128A1503188B2B8C2B55
:10171600942B831203137508FB007608FC007708E8
:10172600FD00831203137508C0007608C100770810
:10173600C2007508BD007608BE007708BF000A1211
:101746008A150B200A128A15831203133D08A60078
:101756003E08A7003F08A8007508C0007608C1002B
:101766007708C2007508BD007608BE007708BF007E
:101776000A128A150B200A128A15831203133D08D2
:10178600A9003E08AA003F08AB007B08C0007C0801
:10179600C1007D08C2007B08BD007C08BE007D0834
:1017A600BF000A128A150B200A128A158312031328
:1017B6003D08A3003E08A4003F08A5002308C0007A
:1017C6002408C1002508C2002908BD002A08BE0059
:1017D6002B08BF000A168A1187200A128A1583125F
:1017E60003133D08B2003E08B3003F08B4003208B8
:1017F600BD003308BE003408BF007808C000790871
:10180600C1007A08C2000A128A150B200A128A152C
:10181600831203133D08AF003E08B0003F08B10035
:101826002F08BD003008BE003108BF007808C00090
:101836007908C1007A08C2000A128A150B200A121A
:101846008A15831203133D08AC003E08AD003F081D
:10185600AE002C08BD002D08BE002E08BF000030CB
:10186600C0007A30C1004430C2000A128A150B202B
:101876000A128A15831203133D08B5003E08B60006
:101886003F08B7007808C0007908C1007A08C2008E
:101896007808BD007908BE007A08BF000A128A15CA
:1018A6000B200A128A15831203133D08C0003E0856
:1018B600C1003F08C2002608BD002708BE00280850
:1018C600BF000A168A1187200A128A15831203138B
:1018D6003D08BD003E08BE003F08BF007B08C000B3
:1018E6007C08C1007D08C2000A128A150B200A1264
:1018F6008A15831203137B08C0007C08C1007D088B
:10190600C2000A128A150B200A128A1583120313C3
:101916003D08C0003E08C1003F08C2003508BD00B2
:101926003608BE003708BF000A168A1173240A1249
:101936008A15831203133D08BA003E08BB003F0810
:10194600BC003A08C0003B08C1003C08C200C030D9
:10195600BD007930BE004430BF000A168A115F21EF
:101966000A128A150318B82CB92C4D2D83120313AD
:101976003A08C0003B08C1003C08C200E630BD0082
:101986007330BE004930BF000A168A115F210A1261
:101996008A150318CF2CD02C2B2D831203133A084B
:1019A600C0003B08C1003C08C2002E30BD006E30AE
:1019B600BE004E30BF000A168A115F210A128A1530
:1019C6000318E62CE72C092D831203136B30C00095
:1019D6006E30C1004E30C2003A08BD003B08BE0062
:1019E6003C08BF000A168A1173240A128A1583124C
:1019F60003133D08BA003E08BB003F08BC00043094
:101A06000A168A11FA240A128A152A2D831203133A
:101A16002430C0007430C1004930C2003A08BD000D
:101A26003B08BE003C08BF000A168A1173240A123E
:101A36008A15831203133D08BA003E08BB003F080F
:101A4600BC0005300A168A11FA240A128A154C2D92
:101A5600831203130030C0007A30C1004430C20044
:101A66003A08BD003B08BE003C08BF000A168A11B2
:101A760073240A128A15831203133D08BA003E081E
:101A8600BB003F08BC0006300A168A11FA240A1267
:101A96008A15532D07300A168A11FA240A128A1556
:101AA600831203130030C000C830C1004230C200A8
:101AB6003A08BD003B08BE003C08BF000A128A1562
:101AC6000B200A128A15831203133D08BA003E083A
:101AD600BB003F08BC003A08BD003B08BE003C08FE
:101AE600BF000A168A1111230A128A1583120313DC
:101AF6003D08B801B8073E08B901B9073808BD0165
:101B0600BD073908BE01BE070A128A15C4210A128A
:101B16008A1508000530C8000030C90007300A12CF
:101B26008A11DE270A128A15A63083120313C00013
:101B36000730C1000A128A11BB200A128A150A163A
:101B46008A11FA230A128A15831203133D08AF017C
:101B5600AF073E08B001B0072F08BD01BD0730082A
:101B6600BE01BE070A168A11CE200A128A158312F2
:101B760003133D08FB003E08FC003F08FD007B0800
:101B8600C0007C08C1007D08C2007508BD0076084B
:101B9600BE007708BF000A168A115F210A128A154D
:101BA6000318D62DD72DDF2D831203137508FB00DE
:101BB6007608FC007708FD00831203137508C00041
:101BC6007608C1007708C2007508BD007608BE0019
:101BD6007708BF000A128A150B200A128A1583128B
:101BE60003133D08A9003E08AA003F08AB0075088C
:101BF600C0007608C1007708C2007508BD007608E7
:101C0600BE007708BF000A128A150B200A128A1531
:101C1600831203133D08AC003E08AD003F08AE003A
:101C26007B08C0007C08C1007D08C2007B08BD009F
:101C36007C08BE007D08BF000A128A150B200A1216
:101C46008A15831203133D08A3003E08A4003F082B
:101C5600A5002308C0002408C1002508C2002C08DE
:101C6600BD002D08BE002E08BF000A168A11872067
:101C76000A128A15831203133D08A6003E08A70020
:101C86003F08A8007808C0007908C1007A08C20099
:101C96007808BD007908BE007A08BF000A168A11C6
:101CA60087200A128A15831203133D08C0003E08D6
:101CB600C1003F08C2002908BD002A08BE002B0843
:101CC600BF000A168A1187200A128A158312031387
:101CD6003D08C0003E08C1003F08C2002608BD00FE
:101CE6002708BE002808BF000A128A150B200A1210
:101CF6008A15831203134030C0001C30C1004630E1
:101D0600C2000A128A150B200A128A1583120313BF
:101D16003D08B4003E08B5003F08B6007508C0008F
:101D26007608C1007708C2007508BD007608BE00B7
:101D36007708BF000A128A150B200A128A15831229
:101D460003137808C0007908C1007A08C2000A1295
:101D56008A150B200A128A15831203137808C0000D
:101D66007908C1007A08C2000A128A150B200A12E5
:101D76008A15831203137B08C0007C08C1007D0806
:101D8600C2000A128A150B200A128A15831203133F
:101D96007B08C0007C08C1007D08C2000A128A15B3
:101DA6000B200A128A15831203133630C0001A302C
:101DB600C1004730C2000A128A150B200A128A1582
:101DC600831203133D08B1003E08B2003F08B3007A
:101DD6003108C0003208C1003308C2003408BD0013
:101DE6003508BE003608BF000A168A1173240A1287
:101DF6008A15831203133D08BD003E08BE003F0846
:101E0600BF006030C0006330C1005830C2000A1203
:101E16008A150B200A128A15831203133D08B70090
:101E26003E08B8003F08B9003708C0003808C100AE
:101E36003908C200C030BD007930BE004430BF0052
:101E46000A168A115F210A128A1503182B2F2C2FC6
:101E5600C02F831203133708C0003808C1003908A1
:101E6600C200E630BD007330BE004930BF000A161E
:101E76008A115F210A128A150318422F432F9E2FBB
:101E8600831203133708C0003808C1003908C2009E
:101E96002E30BD006E30BE004E30BF000A168A11CD
:101EA6005F210A128A150318592F5A2F7C2F831285
:101EB60003136B30C0006E30C1004E30C2003708CD
:101EC600BD003808BE003908BF000A168A117324FF
:101ED6000A128A15831203133D08B7003E08B8009C
:101EE6003F08B90000300A168A11FA240A128A1528
:101EF6009D2F831203132430C0007430C100493073
:101F0600C2003708BD003808BE003908BF000A16EF
:101F16008A1173240A128A15831203133D08B70027
:101F26003E08B8003F08B90001300A168A11FA24A3
:101F36000A128A15BF2F831203130030C0007A30AD
:101F4600C1004430C2003708BD003808BE00390859
:101F5600BF000A168A1173240A128A158312031304
:101F66003D08B7003E08B8003F08B90002300A161F
:101F76008A11FA240A128A15C62F03300A168A1104
:101F8600FA240A128A15831203130030C000C830DF
:101F9600C1004230C2003708BD003808BE0039080B
:101FA600BF000A128A150B200A128A158312031320
:101FB6003D08B7003E08B8003F08B9003708BD0025
:101FC6003808BE003908BF000A168A1111230A1202
:101FD6008A15831203133D08AF01AF073E08B0010F
:101FE600B0072F08BD01BD073008BE01BE070A12A3
:0A1FF6008A15C4210A128A1508009A
:1020A6004130CC00EE30CB00CB0B5728CC0B572859
:1020B6006400831203130130C9020030031CCA03F3
:1020C600CA024A084904031D69286A2853280800D9
:1020D6000530831603139C00CF3085008116011648
:1020E60081110115811401140A168A1185230A1615
:1020F6008A110A168A11F8200A168A118316031302
:1021060006140710811308008030C2064008C60076
:102116004108C7004208C8003D08C3003E08C40085
:102126003F08C5000A128A11E0200A168A11831296
:1021360003134308BD004408BE004508BF00A3289A
:1021460008000030CC000030CD00481CAB28AC287D
:10215600B2284A08CC070318CD0A4B08CD07013030
:102166000310CA0DCB0DFF3E031DB328013003102B
:10217600C90CC80CFF3E031DBA2849084804031DB4
:10218600C528C628A8284C08C801C8074D08C90193
:10219600C907CD2808003E083D04031DD328D428CE
:1021A600DB280030BD000030BE000030BF00F7283D
:1021B6003D08C3003E08C400C5014308C0004408EA
:1021C600C1004508C2008E30CF0040300A168A1181
:1021D60045260A168A11831203134008BD004108DA
:1021E600BE004208BF00F728080000308312031320
:1021F600C8000030C90000300A128A11DE270A160C
:102206008A11003083120313A5000030A6000B29A3
:10221600CB010314CB0D00300A168A11AC220A1624
:102226008A11831203130130A5070318A60A00308A
:10223600A60701302602031D2229F8302502031CB9
:10224600252926290B2908004308420403192C29AD
:102256002D295D29C4010314C40D3C290130031046
:10226600C20DC30DFF3E031D32290130C5004508CE
:10227600C407C31F3F294029312943084102031DD2
:10228600462942084002031C49294A295029420886
:10229600C0024308031CC103C10201300310C30C72
:1022A600C20CFF3E031D51290130C402031D5C29E7
:1022B6005D2940295E290800BF1F62296329792903
:1022C6000030C3000030C4008030C5003D08C302A2
:1022D6003E080318C403C4023F080318C503C50219
:1022E6004308BD004408BE004508BF00C21F7C2944
:1022F6007D2993290030C3000030C4008030C5001A
:102306004008C30241080318C403C4024208031864
:10231600C503C5024308C0004408C1004508C20001
:102326008030BF068030C20642083F02031DA12945
:1023360041083E02031DA12940083D020318A429B5
:10234600A6290314A7290310A82908000030C500F0
:102356000030C600430842040319B229B329EB2909
:10236600C4010314C40DC22901300310C20DC30DEC
:10237600FF3E031DB8290130C7004708C407C31F25
:10238600C529C629B72901300310C50DC60DFF3E64
:10239600031DC72943084102031DD32942084002F1
:1023A600031CD629D729DE294208C0024308031C8C
:1023B600C103C102451401300310C30CC20CFF3E19
:1023C600031DDF290130C402031DEA29EB29C629B2
:1023D6004508C001C0074608C101C107F229080027
:1023E600D0005008840083130008D200840A000835
:1023F600D300840A0008D4000F300310D40CD30C89
:10240600D20CFF3E031D002A5208D100D5004F080A
:10241600840055088000D108031D122A132A1F2A9A
:102426005008840000308000840A00308000840A4E
:102436000030800000304C2A0310003003180130B1
:10244600D1005008840000308004840A8030800463
:10245600840A00308004500884000008D200840AF0
:102466000008D300840A0008D400D41F3B2A3C2A63
:10247600402A0130D2005208D10750088400FF30AC
:102486008005840AFF308005840A003080055108E3
:102496004C2A080083120313A300A308031D542A21
:1024A600962A0430C8000030C90046300A128A1144
:1024B600DE270A168A1183120313CB010314CB0DF0
:1024C6001C300A168A11AC220A168A1183120313CB
:1024D600CB010314CB0D3E300A168A11AC220A1624
:1024E6008A1183120313CB010314CB0D36300A165F
:1024F6008A11AC220A168A1183120313CB01031424
:10250600CB0D3E300A168A11AC220A168A118312A6
:102516000313CB010314CB0D1C300A168A11AC220F
:102526000A168A11AB2A0430C8000030C9004630AA
:102536000A128A11DE270A168A11D530831203136E
:10254600C0000730C1000A128A11BB200A168A1180
:102556000800CC008714CB08031DB22AB32AB42A7C
:102566008710000007110000871200000712CC1F19
:10257600BD2ABE2ABF2A071600008716000087124A
:10258600000007124C1FC82AC92ACA2A07160000CB
:1025960087160000871200000712CC1ED32AD42A01
:1025A600D52A0716000087160000871200000712BA
:1025B6004C1EDE2ADF2AE02A0716000087160000D6
:1025C600871200000712CC1DE92AEA2AEB2A071611
:1025D6000000871600008712000007124C1DF42A1F
:1025E600F52AF62A07160000871600008712000053
:1025F6000712CC1CFF2A002B012B0716000087169A
:1026060000008712000007124C1C0A2B0B2B0C2B08
:102616000716000087160000071508004230CF0095
:102626003D300A168A11F3210A168A118312031302
:10263600C1003D08C3003E08C4003F08C500C601EE
:102646008E30C202C21F282B292B4C2B4208831323
:10265600803A8F3E0318302B312B3A2B0030C000C6
:102666000030BF000030BE000030BD00842B0130BA
:102676000310C60CC50CC40CC30CFF3E031D3B2B3C
:102686000130C7004708C207031D4A2B4B2B3A2BC4
:102696006C2B20304202031C512B522B5B2B00303B
:1026A600C0000030BF000030BE000030BD00842BEB
:1026B600672B0130C7000310C30DC40DC50DC60D31
:1026C600C70B5E2B0130C202C208031D6B2B6C2B9D
:1026D6005C2BC108031D702B7B2BC309C409C509DC
:1026E600C609C30A0319C40A0319C50A0319C60A87
:1026F6004608C0004508BF004408BE004308BD00A8
:10270600842B080003100030031801308700831261
:1027160003138230A400DD30A300A30B902BA40B7F
:10272600902B952B000083120313871200000716C7
:102736000000871000000715000087118230A400F2
:10274600DD30A300A30BA52BA40BA52BAA2B83126C
:10275600031387150310003003180130CB00213016
:102766000A168A11AC220A168A1103108312031361
:10277600003003180130CB00C8300A168A11AC228B
:102786000A168A110310831203130030031801304E
:10279600CB0006300A168A11AC220A168A110310DB
:1027A60083120313003003180130CB0013300A16CE
:1027B6008A11AC220A168A11031083120313003001
:1027C60003180130CB0020300A168A11AC220A16F3
:1027D6008A11031083120313003003180130CB0053
:1027E6000C300A168A11AC220A168A1108008312C6
:1027F60003130B11831603130512023083120313FE
:10280600C9000030CA000A168A1153200A168A1116
:1028160003108312031300300318013081000A30BD
:10282600C9000030CA000A168A1153200A168A11F6
:10283600831603130516831203130108C300C4018C
:102846004308BF004408C0000030C1000030C20089
:102856008316031301160000000001120000000099
:10286600831203130130C1070318C20A0030C207DE
:102876000108C300C40140084406031D442C3F0858
:102886004306031D472C482C522C01304202031DDF
:102896004E2C00304102031C512C522C2B2C0030A4
:1028A600C3000130C40041084302C5004208031CAE
:1028B600420A4402C6004008C8003F08C700083064
:1028C60084000310C70DC80D840B642C4508470708
:1028D600BD0046080318460A4807BE00722C0800C9
:1028E6000030C7000030C8000030C9004530CF00B6
:1028F6003D300A168A11F3210A168A118312031330
:10290600C400C508031D882C892C902C4708BD00DF
:102916004808BE004908BF00F92C4330CF004030BC
:102926000A168A11F3210A168A1183120313C600A6
:10293600C308031D9F2CA02CA72C4708BD004808E0
:10294600BE004908BF00F92C43088313893ECA001C
:102956004A08C5024608CA004A08C4061830C60016
:1029660001300310C70DC80DC90DFF3E031DB42C61
:1029760042083F02031DC52C41083E02031DC52C1B
:1029860040083D02031CC82CC92CD42C4008BD02AB
:102996004108031C410FBE024208031C420ABF0243
:1029A600471401300310BD0DBE0DBF0DFF3E031DC4
:1029B600D52C0130C602031DE12CE22CB32C4508B0
:1029C6008313CF0047300A168A1145260A168A1144
:1029D60083120313C408031DF12CF22CC9174708F0
:1029E600BD004808BE004908BF00F92C0800831244
:1029F6000313BD000230C8000030C9003C300A1283
:102A06008A11DE270A168A11031083120313003077
:102A160003180130BE000F2D2430CA000030CB0051
:102A26003D088313BF00C0013F08C8004008C90025
:102A36000A168A11A4200A168A11831203133E0865
:102A46004807C1000030031801304907C200CB30E7
:102A56004107840005300318063042070A128A111E
:102A660000220A168A11CB010314CB0D0A168A110D
:102A7600AC220A168A11013083120313BF003F08E5
:102A8600BE0712303E02031C492D4A2D0F2D03307E
:102A9600C8000030C9003C300A128A11DE270A1627
:102AA6008A11123083120313BE00592D2430CA0036
:102AB6000030CB003D088313BF00C0013F08C800AB
:102AC6004008C9000A168A11A4200A168A11831220
:102AD60003133E084807C1000030031801304907B8
:102AE600C200CB3041078400053003180630420788
:102AF6000A128A1100220A168A11CB010314CB0D81
:102B06000A168A11AC220A168A110130831203139F
:102B1600BF003F08BE0724303E02031C932D942DB0
:102B2600592D0800C20001304202031C9B2D9C2D2A
:102B3600A22D06304202031CA12DA22DA32D442E48
:102B46004B304002031CA82DA92DAA2D442E0A3075
:102B56004102031CAF2DB02DB12D442EFF30C40011
:102B6600FF30C500420883134407C8004508031810
:102B7600450AC90040080A128A11DE270A168A1178
:102B8600031083120313003003180130C300CB2D4A
:102B9600CB010314CB0D41088313C400C5010430D7
:102BA60084000310C40DC50D840BD42D43084407BF
:102BB600C6000030031801304507C700EB30460752
:102BC600840006300318073047070A128A110022CC
:102BD6000A168A110A168A11AC220A168A110130BF
:102BE60083120313C4004408C30708304302031CBE
:102BF600FD2DFE2DCB2D42088313C400C5014408CC
:102C0600C8004508C90040080A128A11DE270A16BC
:102C16008A11083083120313C300112ECB0103144B
:102C2600CB0D41088313C400C50104308400031092
:102C3600C40DC50D840B1A2E43084407C600003088
:102C4600031801304507C700EB30460784000630FD
:102C56000318073047070A128A1100220A168A113A
:102C66000A168A11AC220A168A110130831203133E
:102C7600C4004408C30710304302031C432E442EED
:102C8600112E0800D000CF08031D4A2E5C2E5008D6
:102C9600840083130008D100840A0008D200840A45
:102CA6000008D300530852045104031D5B2E5C2E0A
:102CB600682E50088400003083138000840A003098
:102CC6008000840A003080001A2F7B2E0130D1004C
:102CD6005108CF07500884000130D100840A840AC5
:102CE6000310800C8403800C8403800CD10B712E9E
:102CF6000030D1000030D200FE30D30050088400EE
:102D06000008D400840A0008D500840A0008D6000A
:102D16005408D1055508D2055608D3055308520460
:102D26005104031D972E982E692EBA2E0130D1001C
:102D36005108CF075008840001308007840A00300C
:102D46000318013E031D8007840A00300318013E64
:102D56008007500884000130D100840A840A0310D9
:102D6600800C8403800C8403800CD10BB02E0030C1
:102D7600D1000030D200FF30D30050088400000894
:102D8600D400840A0008D500840A0008D600540836
:102D9600D1055508D2055608D305530852045104E7
:102DA600031DD62ED72E992EE62E0130CF025008BF
:102DB60084000130D1000310800D840A800D840A3E
:102DC600800DD10BDE2E500884000008D100840A45
:102DD6000008D200840A0008D300D21FF32EF42E76
:102DE600D82E4F18F72EF82E022F50088400FF30E9
:102DF6008005840A7F308005840AFF308005031031
:102E0600CF0C4F08D100D201D30110300310D10DE1
:102E1600D20DD30DFF3E031D092F50088400510823
:102E26008004840A52088004840A53088004080037
:102E36000A168A11F8200A168A1101308312031322
:102E4600C8000030C90001300A128A11DE270A16AE
:102E56008A11B33083120313C0000730C1000A126F
:102E66008A11BB200A168A11033083120313C80085
:102E76000030C90001300A128A11DE270A168A11AB
:102E8600983083120313C0000730C1000A128A115A
:102E9600BB200A168A118312031307100A168A1119
:102EA600FA230A168A11831203133D08BD01BD07D2
:102EB6003E08BE01BE070A168A11CE200A168A11DE
:102EC600831203133D08F5003E08F6003F08F7009D
:102ED6003230C9000030CA000A168A1153200A1679
:102EE6008A110A168A11FA230A168A118312031303
:102EF6003D08BD01BD073E08BE01BE070A168A1180
:102F0600CE200A168A11831203133D08F5003E08E7
:102F1600F6003F08F70007140A168A11FA230A1664
:102F26008A11831203133D08BD01BD073E08BE0189
:102F3600BE070A168A11CE200A168A1183120313B7
:102F46003D08F8003E08F9003F08FA003230C90093
:102F56000030CA000A168A1153200A168A110A1668
:102F66008A11FA230A168A11831203133D08BD013A
:102F7600BD073E08BE01BE070A168A11CE200A16F4
:102F86008A11831203133D08F8003E08F9003F0832
:102F9600FA0007100430C8000030C90000300A12D9
:102FA6008A11DE270A168A110310831203130030D2
:102FB60003180130A300DF2FCB010314CB0DFC3027
:102FC6000A168A11AC220A168A11023083120313DA
:102FD600C9000030CA000A168A1153200A168A113F
:102FE600013083120313A4002408A30754302302DC
:0A2FF600031CFE2FFF2FDF2F080041
:02400E00F23F7F
:00000001FF
